:020000040000FA
:10000000E8270020F90200000103000003030000BC
:1000100005030000070300000903000000000000C2
:100020000000000000000000000000000B030000C2
:100030000D030000000000000F030000110300008A
:100040001303000013030000E10800006D05000029
:100050001303000013030000A103000013030000BA
:100060001303000013030000130300001303000038
:100070001303000013030000130300001303000028
:1000800013030000490500001303000013030000E0
:10009000C105000013030000130300001303000058
:1000A00013030000130300001303000013030000F8
:1000B0001303000013030000000000000000000014
:1000C00013030000130300001303000013030000D8
:1000D00013030000130300001303000000000000DE
:1000E0000000000000000000000000000000000010
:1000F0000000000000000000000000000000000000
:1001000000000000000000000000000000000000EF
:1001100000000000000000000000000000000000DF
:1001200000000000000000000000000000000000CF
:1001300000000000000000000000000000000000BF
:1001400000000000000000000000000000000000AF
:10015000000000000000000000000000000000009F
:10016000000000000000000000000000000000008F
:10017000000000000000000000000000000000007F
:10018000000000000000000000000000000000006F
:10019000000000000000000000000000000000005F
:1001A000000000000000000000000000000000004F
:1001B000000000000000000000000000000000003F
:1001C000000000000000000000000000000000002F
:1001D000000000000000000000000000000000001F
:1001E000000000000000000000000000000000000F
:1001F00000000000000000000000000000000000FF
:10020000DFF80CD000F0BAF8004800474D100000AD
:10021000E827002030B4044654E8000F0D4644E8B7
:100220000053002BF8D1156030BC704730B4044641
:1002300054E8000F40EA010544E80053002BF7D1D1
:10024000156030BC704730B4044654E8000F00EA33
:10025000010544E80053002BF7D1156030BC70470E
:1002600030B4044654E8000F80EA010544E8005326
:10027000002BF7D1156030BC704730B4044654E809
:10028000000F00EB010544E80053002BF7D1156087
:1002900030BC704730B4044654E8000FA0EB0105B1
:1002A00044E80053002BF7D1156030BC704770B4A0
:1002B00004464FF0000054E8006F0D68AE4207BFDF
:1002C00044E80023012044E800630E60002B1CBFBB
:1002D0000020F0E770BC704730B4044654E8000FCB
:1002E00088422CBF451A054644E80053002BF5D13F
:1002F000156030BC7047000006488047064800473C
:10030000FEE7FEE7FEE7FEE7FEE7FEE7FEE7FEE7C5
:10031000FEE7FEE7C5050000010200000048704747
:10032000E82F000040EA01039B0703D009E008C959
:10033000121F08C0042AFAD203E011F8013B00F8AA
:10034000013B521EF9D27047D2B201E000F8012BF6
:10035000491EFBD270470022F6E710B513460A4645
:1003600004461946FFF7F0FF204610BD421C10F866
:10037000011B0029FBD1801A70470000064C074D75
:1003800006E0E06840F0010394E807009847103465
:10039000AC42F6D3FFF738FF90300000B0300000D9
:1003A0002DE9F04700268AB0DFF85091B0464FF4AF
:1003B0008075012437460696284601F0D7F938B1F2
:1003C000D9F80403204203D0284601F0C5F926439A
:1003D0002D1D64007F1CADB2082FEDD34FF4BE7409
:1003E000204601F0C3F948B1204601F0B5F946F0C6
:1003F000004606AA0121002001F09AF9404D16F0AE
:10040000FF0F15D00127002437420DD009EB8401DE
:10041000D1F81005D1F81015C0F3042055F82420A8
:10042000C1F3014102B190477F00641C082CEBD35B
:10043000002E5FDA4FF0FF30CDF8108054E028191D
:1004400010F8507F90F9000027F0C008401C3BD006
:1004500007A9404600F034FF10B34FEA9719404611
:1004600000F0E8FB55F820701FB1B9F1030F03D07D
:1004700006E0B9F1030F27D104A9404600F028FF98
:100480004FF0A04101EB8800D0F8000706A9C0F3A7
:10049000014A404600F014FF18B1BAF1020F03D030
:1004A00012E0BAF1030F0FD1B9F1030F08D1BAF17D
:1004B000020F1DD00221404601F010F9761CF6B261
:1004C00017B149464046B847641C042CB7D3002EE8
:1004D00010D06A460121002001F02AF906990098FF
:1004E000884207D006900498002634460790A6E775
:1004F0000321E0E70AB0BDE8F0870000006000409B
:10050000E800002000F01F02012191404009800016
:1005100000F1E020C0F88012704700F01F020121B6
:1005200091404009800000F1E020C0F800117047C0
:1005300000F01F02012191404009800000F1E020FD
:10054000C0F800127047000007480021C0F84011B1
:10055000C0F84411C0F84811C0F84C11C0F800119F
:10056000C0F8041102F094BA00100140F8B5124826
:10057000124E04464FF48C7101F0AFFC00281AD0E3
:100580000025C4F81851D4F818010090F07F3446C3
:10059000FF2806D0A17F11B101F0B1F801E001F010
:1005A000B5F865772572D4E9002101B004F108009F
:1005B000BDE8F0401047F8BD003000404401002085
:1005C00002F0D8B9F0B5B5480023021D0178101D1E
:1005D00001254FF0805406290BD11678360708D133
:1005E0000678C6F30316032E06D0042E04D0052E7B
:1005F00002D0062907D00EE0B4F82463A84FC6F352
:1006000004263E6002E01678360704D10678C6F369
:100610000316032E02D0062904D00FE0A24FA14EEC
:100620007E670EE01678360708D10678C6F3031603
:10063000032E06D0042E04D0052E02D0062907D0A2
:100640000EE0D4F84462994FC6F342363E6002E0B1
:100650001678360704D10678C6F30316032E02D0A7
:10066000062906D011E0924E376827F08077376070
:100670000EE01678360708D10678C6F30316032E67
:1006800006D0042E04D0052E02D006290AD011E08F
:100690004FF08046C6F80C31C6F81031834E361F35
:1006A000336002E01678360704D10678C6F30316E5
:1006B000032E02D0062905D00CE07C4F03266437B8
:1006C0003E600AE01678360704D10678C6F30316B2
:1006D000032E02D006290DD014E0764F05263E6089
:1006E000744E78363560734E083633603F263F1DB2
:1006F0003E6002E01678360704D10678C6F303168A
:10070000052E02D0062957D062E06B4E36686B4F3B
:100710003E60694E361D36683F1D3E60664E0836A7
:1007200036683F1D3E60644E0C3636683F1D3E60A5
:10073000614E103636683F1D3E605F4E1436366897
:100740003F1D3E605C4E183636685C4F20373E6079
:10075000594E1C3636683F1D3E60574E203636686F
:100760003F1D3E60544E243636683F1D3E60524E5B
:10077000283636683F1D3E604F4E2C3636683F1D8A
:100780003E604D4E303636684C4F40373E604A4EE4
:10079000343636683F1D3E60474E383636683F1D5A
:1007A0003E60454E3C3636683F1D3E60424E403608
:1007B00036683F1D3E6002E01678360708D106789D
:1007C000C6F30316032E06D0042E04D0052E02D045
:1007D000062907D019E0D4F85812394A01F04F0120
:1007E000116002E0117809070FD10078C0F30310FF
:1007F000032803D0042801D0052806D13148016818
:10080000C90702D06FF001010160D4F83001062859
:1008100008D1D4F83401062804D12B48016841F4EA
:100820008061016022487438016841F47001016000
:10083000BFF34F8FBFF36F8F4FF01021D1F800023D
:10084000002803DBD1F80402002822DA1F4A1560D1
:100850001F480468002CFCD01524C1F8004205682C
:10086000002DFCD0C1F8044201680029FCD01360BF
:1008700001680029FCD0BFF34F8F0D48F0380168A4
:10088000144A01F4E06111430160BFF34F8F00BFD0
:10089000FDE7124910480860F0BD0000E00F00F0CD
:1008A000403501400DF0ADBA00C007403C050040A6
:1008B000FCED00E0105600400404001020C500408C
:1008C000E40E0040000400403C17004004E50140F5
:1008D00000E401400400FA050090D003B0000020BD
:1008E00001480068004700001C00002002E008C822
:1008F000121F08C1002AFAD170477047002001E09A
:1009000001C1121F002AFBD17047000072B601F02E
:100910000BFA00BF01F00AF80028FBD1104C0121AE
:10092000208801EB00400FA101F060F91048006839
:10093000C00700D000BE2088022101EB00400DA1BD
:1009400001F054F9BFF34F8F0948E43801680D4AAC
:1009500001F4E06111430160BFF34F8F00BFFDE779
:10096000CC000020466174616C206572726F720069
:10097000F0ED00E053797374656D207265736574F2
:10098000000000000400FA050EB500210091CDE939
:1009900001106A4644F20100FFF7B8FF0EBD00F0F7
:1009A00003B800F009B8000072B602480168491C9B
:1009B000016070473800002003490868401E086045
:1009C00000D162B670470000380000202DE9F041E8
:1009D000064608680C46411C4FF0A0474FF0010541
:1009E00006D005FA00F1C7F80815206800F062FE8D
:1009F0006068411C02D0002100F040FE3168A0690F
:100A0000C1F82405607D227D31681043C1F86C0572
:100A1000D4E900123068C0F81425C0F80C15207D08
:100A2000012815D1A068411C02D0002100F026FE4B
:100A3000E068411C05D08540C7F80855E06800F023
:100A400039FED4E902123068C0F80825C0F8101544
:100A5000BDE8F0812DE9F041064608680C46411CCE
:100A60004FF0A0474FF0010506D005FA00F1C7F896
:100A70000815206800F028FE6068411C02D00021A3
:100A800000F005FE3168A069C1F82405607D217D74
:100A900032680843C2F86C05D4E900123068C0F827
:100AA0000C15C0F81425207D012815D1A068411C23
:100AB00002D0002100F0EBFDE068411C05D085402C
:100AC000C7F80855E06800F0FFFDD4E9021230686D
:100AD000C0F80825C0F81015BDE8F0812DE9FC41EB
:100AE0000646C0074FF000050ED0104F002401222B
:100AF000385D009500231146019500F065FD641CEA
:100B0000042CF4D300F02EF8B0070DD5074E0024C6
:100B1000361D0022305D032300951146019500F03B
:100B200053FD641C042CF4D3BDE8FC81F82E0000B6
:100B300007490B5C4FF0A041D1F8042501209840F3
:100B400020EA0203C1F808351040C1F80C057047CF
:100B5000F82E00000249085C012100F0DEBD000013
:100B6000F82E000010B500242046FFF7F3FF641CA8
:100B7000042CF9D310BD00002DE9F0470546861C72
:100B800090460F464FF001090020FFF708FF1B4C6D
:100B900020683860D4E90001401AA16804F21C47BB
:100BA000081A0EE00121384600F022FB00F000FA9E
:100BB0000146384600F01CFBD4E90001401AA16848
:100BC000081A401C8642EDD8B8F1000F03D005206A
:100BD00065F3891002E0062065F39F50A268216842
:100BE000114004EB8101C86020683044206000207F
:100BF000FFF7D7FE4846BDE8F0870000C403002099
:100C000030B482680468531C8360A154D0E9011297
:100C10008A4202D330BC00F0DEBB30BC704700001B
:100C2000034803C8814201D101207047002070476A
:100C3000C40300200249084490F9300070470000C6
:100C4000E80000202DE9F05F26484168F1B3DFF8A5
:100C500098B00E688146DBF8004087688078E11B19
:100C600021F07F45ED1CB0B9DFF880804FF4803073
:100C7000C8F84403C8F804031120FFF743FC11200F
:100C8000FFF74BFC4FF0010AC8F800A02F2001F03D
:100C900045F989F802A0B54200D23546124BE81951
:100CA0003C3320F07F401860DBF800105A46091BE7
:100CB00021F07F41001B20F07F40C91C81420FD9E9
:100CC000106818602F2001F029F900E004E0BDE869
:100CD000F05F1120FFF72CBCBDE8F05F01F0E2BC33
:100CE000BDE8F09F240000200415014000100140E1
:100CF00010B50021024800F086FA80F3100010BD04
:100D0000E00700200E4910B50A784C780023A24273
:100D100012D0521CD2B20A70022A00D10B70084ABB
:100D20000B780C3252F8232002608868104420F0BF
:100D30007F408860012010BD0360002010BD0000CE
:100D4000240000202DE9FC5F0E008346DDE90C47FE
:100D5000C6F1000098469246814600D40846012517
:100D600003E000BF90FBFAF06D1C5045FADAA8458D
:100D700000D9454624B1002E01DB780700D5641E5A
:100D8000B80702D5B8F1000F0AD0F80708D13CB176
:100D9000A54205D220215846641EFFF731FFF6E731
:100DA000002E02DA4E462D2102E0780703D52B21D2
:100DB0005846FFF725FF07F0030002280BD1B8F1D2
:100DC000000F08D13CB1A54205D230215846641E1F
:100DD000FFF716FFF6E7CDE9004743465246314696
:100DE000584602F019F8BDE8FC9F000070B50D46AA
:100DF000044600684FF4887101F08AF84FF490714E
:100E0000206801F085F84FF49271206801F080F8B5
:100E10004FF4A271206801F07BF820681249C0F8F5
:100E2000041320686907000B40B2090E002806DA97
:100E300000F00F0000F1E02080F8141D03E000F145
:100E4000E02080F8001420680121000B40B200F07F
:100E50001F0291404009800000F1E020C0F880129C
:100E6000C0F8001170BD000010030200024600200F
:100E70001268930702D0530702D47047500714D565
:100E800002F00300012802D002280CD105E0C2F3D1
:100E900083100B68801C184404E00223086803EBED
:100EA00092521044086001207047086800EB92538A
:100EB000C2F38910401CEEE72DE9F047394E0027B8
:100EC00080463D46DFF8E090D6F804A057E003D016
:100ED0000446D0F81C8035E099F8002002EB42016E
:100EE000521CD2B289F8002009EBC10199F80230F6
:100EF000091D9A4201D189F8005048680A780446D1
:100F0000012A12D0022A02D0032A3BD108E001F0C4
:100F10008FFD00B10127257434E00574C06900E03D
:100F200070680028F9D170602CE0207C50BB886884
:100F30006060C868A0600869E0604869A061F078F6
:100F400000B165606268B168184B501A20F07F40AC
:100F5000984202D2A168084406E0881AA16820F0ED
:100F60007F40814202D9081A206000E02560656058
:100F70000120A56020742046E56101F03BFDB8F139
:100F80000000A4D199F8001099F801008142A3D182
:100F900017B97168514502D00120BDE8F0870020E3
:100FA000FBE7000024000020B8010020FFFF7F00C5
:100FB0002DE9FF410026234800F017F92148001FC2
:100FC000074600F012F9204C60680090A56800E028
:100FD00000986946284004EB80000C30FFF746FF7C
:100FE0000028F5D101AA009901EA050304EB830367
:100FF000491CDB6842F82030401C00910228F2D3E3
:10100000019800F0030001280BD0022810D10198AC
:10101000032101EB90500099BDF80A6001EB9000AC
:1010200005E00198BDF80A60C0F383100844009001
:10103000384600F0D7F808B10098606004B0304638
:10104000BDE8F081DC070020C40300208EB0012041
:10105000FFF744FD4FF40041002000F021FE08B1ED
:10106000FFF792FC00F054FC2A490DF1100C032408
:101070000FC98CE80F001D208DF813001C208DF87F
:10108000120004208DF8110022488DF81040002332
:10109000214A04A9103800F025F908B1FFF774FCC3
:1010A0001E481FA1008804EB004000F09FFD224C69
:1010B0004FF00008C4F80880A4F80C8084F80E8073
:1010C00084F800801C490722491CCB1D15468DE879
:1010D0002E00104800220C38694601F021F818B1A2
:1010E000FFF752FC00E020BF20780028FBD000BFB3
:1010F00000F01CFC0028FBD1FFF71AFD054DC826A7
:10110000183D4FF47A47691C38468847761EFAD155
:10111000D0E70000E82E000081270000CC0000206E
:10112000535049206578616D706C652073746172ED
:101130007465642E00000000000000202DE9F047D7
:10114000C7880446181D16468946B0FBF7F1B0FB68
:10115000F7F207FB12009A193A44D21CB2FBF7F2DD
:10116000DDF820A001E02468491E0029FBD13D1ACA
:101170008846B54216D818E0BAF1000F05D02118FC
:1011800009EB08002A46091D04E0204409EB080188
:101190002A46001DFFF7C6F800202468761BA844E5
:1011A000B74201D9354600E03D46002EE4D1BDE806
:1011B000F087000030B5024659B100F09DFD0021D6
:1011C000074C09E004EB810315685B88AB4202D150
:1011D0001160002030BD491C8142F3D3052030BD91
:1011E000B4000020002100F009B8012100F010B87F
:1011F00008B56A46FFF741F8009808BD08B56A4689
:10120000FFF721F808BD08B56A46FFF703F808BDE7
:1012100008B56A46FFF70AF8009808BD08B56A469F
:10122000FFF738F8009808BD70B504460025284639
:10123000FFF7B5FB21686268086890420ED9401E2E
:1012400008600178A38AE26801FB0325227A2168FD
:10125000101AC0B20A79824200D208710020FFF74A
:10126000A0FB284670BD70B505460C460020FFF770
:1012700096FBE868A98A201AB0FBF1F12A68106889
:10128000431C13600170BDE870400020FFF789BB6C
:1012900010B530B1017A42680368891AC9B21A6080
:1012A00006E00E2010BD03681A68541C1C60117003
:1012B000491EC9B2F7D2006800210171084610BD6D
:1012C000C20800F007030120895C9840084070477D
:1012D00010B5C20800F00703885C01249C4020433D
:1012E000885410BD2DE9FF411C460378164D174E5A
:1012F00045F823200C3545F82340F0CE8DE8F0006A
:101300000C788DF800404C788DF801408C788DF881
:101310000240CC788DF803400C798DF805404C796B
:101320008DF806408C6802940C7B8DF80C40497B4C
:101330008DF80D1002B1064A6946001D00F028FE26
:1013400004B0BDE8F0810000D0000020002F0000B4
:10135000F5270000F0B505460478154889B0164613
:1013600040F82420124A0869121DA2F1080742F829
:101370002400487F385520226846FEF7D3FF0494A6
:101380002878385C48B10EB10A4A00E0002269466C
:10139000281D01F02DF809B0F0BD0EB1064A00E09D
:1013A0000022694605F10C0000F0F4FEF3E70000AE
:1013B00014000020F52C0000412B00000FB408B5EC
:1013C0000399002904D004AA00926A4600F00FF89D
:1013D00001B05DF814FB10B582680446002A05D000
:1013E000D4E90403216898470020A06010BD2DE9CE
:1013F000FC4791460C00804676D014F8011B39B1A9
:1014000025290ED04046FFF7FBFB20780028F4D1B9
:1014100098F80C00002867D04046BDE8FC47FFF76D
:10142000DABF0020012221782B291BD02D2902D0E0
:10143000302908D102E040F0010001E040F0020054
:10144000641C002AEFD100252A290ED02178A1F1B1
:1014500030020A2A11D205EB850201EB4205641C19
:10146000303DF1E740F00400EAE7D9F800100B1D29
:10147000C9F800300968641C0D44217800232E2926
:101480000BD114F8011FA1F130020A2A05D203EB97
:10149000830201EB4203303BF3E76C290DD068294E
:1014A0000BD0692921D00BDC252918D0582931D03F
:1014B00063290ED0642915D117E014F8011FECE759
:1014C000702969D0732932D075291BD0782909D1A8
:1014D00020E0D9F80000011DC9F80010017840464D
:1014E000FFF78EFB641C90E76CE0D9F800100A1D32
:1014F000C9F800200968CDE900500A224046FFF7EC
:1015000021FCEFE7D9F800100A1DC9F8002009688E
:101510000A2206E0D9F800100A1DC9F8002009685F
:101520001022CDE90050404601F076FCDAE7D9F808
:10153000001000270A1DC9F800200E68C00705D159
:1015400012E04046761C7F1CFFF75AFB31780029D9
:10155000F7D104E0202140466D1EFFF751FBBD424C
:10156000C0D9002DF6D1BDE74EB13046FEF7FEFEE4
:10157000074604E0202140466D1EFFF741FBBD42B7
:1015800006D9002DF6D103E04046761CFFF738FB64
:1015900031780029F8D1A5E7D9F80000011DC9F874
:1015A0000010056830214046FFF72AFB78214046AD
:1015B000FFF726FB08200021CDE900010346102299
:1015C0002946B0E7BDE8FC8770B541EA4201DDE994
:1015D00004564FF0A04441EA830141EA052104EB9F
:1015E000800041EA0641C0F8001770BD70B541EABD
:1015F0004201DDE904564FF0A04441EA830141EA8B
:10160000052104EB800041EA0641C0F8001770BDD7
:1016100070B541EA4201DDE904564FF0A04441EAC9
:10162000830141EA052104EB800041EA0641C0F84C
:10163000001770BD70B541EA4201DDE904564FF074
:10164000A04441EA830141EA052104EB800041EA1C
:101650000641C0F8001770BD1CB5002100910B4673
:1016600001220191FFF7D4FF1CBD1CB500210091A0
:101670000B4601220191FFF7DDFF1CBD1CB50022C6
:101680000B46009211460192FFF7C2FF1CBD1CB52C
:1016900000220B46009211460192FFF7CBFF1CBDC2
:1016A0001CB5002100910B46012201911146FFF764
:1016B0009DFF1CBD1CB5002100910B46012201912C
:1016C0001146FFF7A5FF1CBD1CB5002100910B467C
:1016D000012201911146FFF7ADFF1CBD4FF0A04262
:1016E00002EB8000D0F8002722F44032C0F8002737
:1016F000D0F8002742EA0141C0F8001770474FF0C8
:10170000A04201218140C2F80C1570474FF0A04261
:1017100001218140C2F80815704701224FF0A04313
:10172000824011B1C3F808257047C3F80C257047F3
:1017300018B5084B6C4601441B68009306E000BFD7
:1017400054F82030D3F81035401C08C28142F7D835
:1017500018BD0000102F0000034908B508440021FF
:1017600001600068009008BD0060004002494058D8
:10177000012800D0002070470060004030B5124BB7
:1017800001460020D3F81044224609E0157A85422C
:1017900005D1401C0A28F7DB4FF0FF3030BD5268FE
:1017A000002AF3D1421CF9D00872D3F810242AB1D0
:1017B00052684A60D3F81024516030BD0022C3F84B
:1017C00010144A6030BD0000C4030020F0B595B08D
:1017D0001C4615460F4608461A9E00F05DFB182170
:1017E00009A8FEF7B8FD0E96CDE90954002308229A
:1017F00003A9384600F065FB05980690BDF8100077
:10180000ADF81C00BDF81200ADF81E0000208DF8E8
:1018100021000398082600F00300012802D00228C6
:1018200018D032E003983346850AC0F3C2008DF821
:10183000200003980FA9C0F38314A200384600F0DB
:1018400040FB09A8009006AB22460FA9284600F0ED
:101850007FFA1AE00398840DC0F3C2008DF82000CF
:10186000082C01D2254600E0082533462A460FA958
:10187000384600F026FB2E44641B09AB06AA294615
:101880000FA800F0B7F9002CEAD1384600F00AFBA7
:1018900015B0F0BD7047012001F070B9084810B5CF
:1018A0000178084A515C19B1001D00F02DFE02E0DC
:1018B0000C3000F03BFDBDE81040002001F05EB9A7
:1018C000400000201000002008B5034A0092402389
:1018D000024AFFF77BFF08BD41270000C402002039
:1018E0000A4A012902EBC00007D0022907D00329C8
:1018F00007D0042907D00020704702207047042039
:10190000704700797047407970470000B0300000A0
:1019100010B5FFF7C0FF04210348FFF72FFF02496E
:101920000120487210BD0000540000202DE9F0474E
:101930008CB0FFF775F918B100200CB0BDE8F08746
:10194000784C0020C4F81804BFF34F8F60680290F1
:10195000A5684FF00008284004EB800008E02168EB
:101960000298814201D86160E6E7284004EB8000DC
:101970000C3002A9FFF77AFA0028F0D103AB0299E4
:1019800001EA050204EB8202491CD26843F82020D8
:10199000401C02910228F2D3039800F003000228B1
:1019A00002D001284ED0A5E003985022810D89462F
:1019B000B2EB905F00D850210E4666F39F50039023
:1019C0000831594800F01FFA070078D000F064FA97
:1019D0004346082203A9384600F079FA029908F133
:1019E000080A2940681A8000001D864223D94D4DFF
:1019F0000C3530B1C2B204EB8101301A90460C3183
:101A000004E02946F2B2002590462846C6B2534665
:101A1000384600F05CFA0AEB08032DB1324629463D
:101A20004FEA070000F053FA029909F1030001EBB5
:101A3000900002903AE004EB81015346324638466A
:101A40000C31EFE70398C0F38311062900D3062178
:101A500061F389100390C0F38310801C8100324829
:101A600000F0D1F9070045D000F016FA43460822ED
:101A700003A9384600F02BFA08F1080800260FE009
:101A80000298434600EA0501401C04EB81010290E4
:101A9000042238460C3100F01AFA08F10408761CCA
:101AA0000398C0F38310B042EAD847B1D4F8105479
:101AB000D4F8180468B1384600F0F4F92CE019E0C5
:101AC000687A012804D12A68284639461268904766
:101AD0006D68002DF4D1384600F0E4F90020FEF7DF
:101AE0005EFFD4F8180408B9029860600020FEF781
:101AF00058FF11E0D4F8104404E0216820468968BA
:101B000088476468002CF8D108480221008801EB5E
:101B1000004007A100F06AF8FFF782F880F00100AA
:101B20000BE70000C4030020E8300000CC000020D8
:101B30004261636B656E647320666C75736865647F
:101B4000000000002DE9F84F8146DFF89C80D01C92
:101B500015468A46800800226946D8F80860FFF7D3
:101B60000BF8B8B3009CA01C0090D8F808103040C7
:101B7000091A8F003F1DBD4208EB800002D82A469B
:101B8000514608E03A4651460C30FEF7CBFB16486A
:101B9000EA1B0AEB07010C30FEF7C4FB4FEA1947BA
:101BA000FFF7A6F847EA0042601C304008EB8000CF
:101BB000344008EB8401C260C8684FF6C07269F314
:101BC000C500904365F39F5020F00300801C20F077
:101BD0000400C86098F8200402E000BFFFF7A6FEEA
:101BE0000028FBD1BDE8F88FC403002000231A466B
:101BF00000F07ABE2DE9F0470E4680461C4692461C
:101C000008293ED894F80C900020207319461046FD
:101C100000F0F0FC0025B54206D218F805201AA104
:101C20002046FFF7CBFB03E019A12046FFF7C6FBD8
:101C30006D1C082DEFD317A12046FFF7BFFB002531
:101C4000B54210D218F80570FEF768FB0068C05D59
:101C500010F03E0F01D03A4600E02E220EA12046A1
:101C6000FFF7ACFB03E00DA12046FFF7A7FB6D1CBF
:101C7000082DE5D301222146504600F09DFC84F852
:101C80000C90BDE8F087000020253032780000007D
:101C9000202020007C0000002563000020000000C0
:101CA000104810B5FF218160002101604160C0F83B
:101CB0001814C0F8141480F820140B4800F0F0F841
:101CC00000280DD109480A490A4B401AC1080020D2
:101CD00003E000BF23F82000401C8842FAD3002014
:101CE00010BD0000C4030020E8300000E830000010
:101CF000B0300000B400002002480349401AC00878
:101D000070470000E8300000B030000013B56846AE
:101D1000FFF750FA08B100201CBD0248009950F8A6
:101D200031001CBDB030000070B508480125D0F866
:101D3000104480F8205405E0657221682046496807
:101D400088476468002CF7D170BD0000C4030020F0
:101D50002DE9FF4781460C9D00200C462F7B287300
:101D6000984616462946184600F044FC072E42D2F3
:101D7000DFE806F004090F161F2A360049462846F8
:101D8000FFF71CFB37E0494628462268FFF716FBA1
:101D900031E0D4E9002349462846FFF70FFB2AE04B
:101DA000A0680090D4E9002349462846FFF706FBC7
:101DB00021E0D4E90201CDE90001D4E9002349463C
:101DC0002846FFF7FBFA16E004F1080007C88DE883
:101DD0000700D4E9002349462846FFF7EFFA0AE056
:101DE00004F108000FC88DE80F00D4E9002349462C
:101DF0002846FFF7E3FA00222946404600F0DCFBC4
:101E00002F73BDE8FF872DE9F041858A80462D1F9D
:101E10004819C01CB0FBF5F0C6B24046FFF704FA03
:101E2000041E19D00020207101206071E580002778
:101E30002546761EC4F800800BE04046FFF7F4F913
:101E400060B16179491C6171286005467F1CC0F84A
:101E50000080B742F1D32046BDE8F081204600F073
:101E600002F80020F8E72DE9F041457901466B1EA4
:101E7000002201E00968521C9A42FBD30F68014618
:101E8000002605E038460C68FFF7EDF92146761C80
:101E9000AE42F7D3BDE8F0810121001DFFF7A8B9DC
:101EA000FFF7F6B910B504460121001DFFF7B6F99A
:101EB00010F0FF0F04D12046BDE81040FFF7D3BF5C
:101EC00010BD38B501240094FFF738F938BD38B596
:101ED00000240094FFF732F938BD4058002800D0A4
:101EE000012070474058002800D00120704708B5F5
:101EF000002242504058009008BDD0F8040308402A
:101F000000D0012070474058002800D001207047C1
:101F100008B5002242504058009008BD002802D069
:101F20000149800108477047212F00000121B1EBD2
:101F3000507F01D101207047002070470121B1EB93
:101F4000507F01D1012070470020704770B50D46C9
:101F500000F09CFB04000FD00020FEF720FD20794C
:101F600020B10020FEF71DFD112070BD012025606D
:101F700020710020FEF715FD002070BD10B500F0A7
:101F800085FB002802D000210160017110BD000016
:101F90002DE9FC5F0C4601799046DFF87CB101EB3E
:101FA000C1020BEB82060746307F994610B108202C
:101FB000BDE8FC9F594A3868054652F82110FFF7E2
:101FC000C5FF08B11120F3E7C6E90089207B01288D
:101FD000207802D8FFF793FB01E0FFF797FB4FF063
:101FE000000ACDF800A0CDF804A020785346524650
:101FF0000121FFF7FBFA60784FF0FF38FF2806D089
:102000008146FFF77CFB4846FFF74AFB00E0C146EC
:10201000A078FF2809D0002280460123CDF800A037
:102020001146CDF804A0FFF7E1FA3879A17800EB6A
:10203000C0020BEB820080F82010E078FF2817D058
:10204000217911B1FFF75BFB01E0FFF75FFBE0785F
:10205000FFF726FB3879E17800EBC0020BEB820238
:10206000D1773A79217902EBC2020BEB82008177BA
:102070002278C5F80825C5F80C95C5F81085A06824
:10208000C5F82405217B607B00B10120012904D023
:10209000022905D0032908D105E040F0020004E040
:1020A00040F0040001E040F00600C5F85405A079B6
:1020B000C5F8C005306810B14020C5F804030720FA
:1020C000C5F800053068012108B338686279000B53
:1020D00040B200284FEA421206DA00F00F0000F189
:1020E000E02080F8142D03E000F1E02080F80024C7
:1020F0003868000B40B200F01F0301FA03F24009F8
:10210000800000F1E020C0F88022C0F80021504695
:1021100086F81DA031774BE744010020142F000002
:102120002DE9F04105460F460079154900EBC00046
:1021300001EB80041646607F10B11120BDE8F081EC
:10214000206820B116F0140F01D10120607797E8C4
:102150000F0004F10C0888E80F00E07FFF2806D08C
:10216000A17F11B1FFF7D2FA01E0FFF7C8FA3346B9
:102170003A4621462868BDE8F04100F057BB000010
:10218000440100200149024800F020BD6801002000
:10219000002000402DE9F0410546007916460F4623
:1021A00000EB40012D4A01EBC00102EB810494F8E1
:1021B0002A1011B10820BDE8F081294951F82010FA
:1021C0002868FFF7C3FE08B11120F4E73946284616
:1021D000FEF7FCFB66603869206030004FF00106B6
:1021E0002FD03F7F4FF48E712868FFF780FE4FF4A9
:1021F000A2712868FFF77BFE28681A49C0F804130B
:1022000028684FEA4711000B40B2002806DA00F0B8
:102210000F0000F1E02080F8141D03E000F1E02041
:1022200080F800142868000B40B200F01F0206FA84
:1022300002F14009800000F1E020C0F88012C0F8EF
:10224000001128680421C0F800150020A061E06199
:1022500084F8290044F8140FA675ACE76801002043
:10226000182F0000800002002DE9F0470546007994
:102270000B4600EB400101EBC000234901EB800459
:10228000284600F043F810B11120BDE8F0874FF068
:102290000008C4F82080A360626184F828804FF4AD
:1022A0008E76474631462868FFF721FE28684FF0B2
:1022B0000109C0F808902146286800F023FC6068F6
:1022C00000BBD5F800A00EE094F8280008B10F2755
:1022D00016E031465046FFF705FE0028F4D02146AF
:1022E000504600F00FFC216A60698142F1D331460B
:1022F0002868FFF7F7FD0028F9D02868C0F80C908F
:10230000C4F814803846C0E768010020007900EB6B
:10231000400101EBC000044901EB80004069002846
:1023200000D0012070470000680100202DE9F0472F
:10233000044600794FF0000900EB400101EBC000BA
:10234000254901EB80072068C0F80095786880B1C6
:1023500020682249C0F8081320680121000B40B210
:1023600000F01F0291404009800000F1E020C0F819
:1023700080112068D0F80C25D0F81485D0F80865B5
:10238000D0F810554FF0FF31C0F81415C0F80C15F7
:102390002068C0F80815C0F81015501C02D010466F
:1023A000FFF75AF9B8F1FF3F02D04046FFF754F962
:1023B000681C02D02846FFF74FF9701C02D0304647
:1023C000FFF74AF92068FFF7D9FD87F82A90C7F888
:1023D0000490BDE8F087000068010020840202003C
:1023E0000149024800F09EBC9401002000200040FA
:1023F0002DE9F0410546164600790F46154A00EBD7
:10240000C00102EB810494F8201011B10820BDE84E
:10241000F081114951F820102868FFF797FD08B1A5
:102420001120F4E739462846FEF714FB6660386948
:1024300020601EB1397F2846FEF7D8FC28680821A5
:10244000C0F800150020A061E0610121606184F8FE
:102450002010DCE7940100201C2F00002DE9F0473C
:1024600004460E460079204900EBC00001EB8005D0
:1024700017463046FFF762FD30B1204600F036F8CF
:1024800020B11120BDE8F0871020FBE76F61AE603E
:102490004FF49076002731462068FFF739FD4FF45E
:1024A000AC7841462068FFF733FD2068AA68696967
:1024B000C0F84425C0F8481520680121816068688B
:1024C00078B9B14649462068FFF71DFD06464146EA
:1024D0002068FFF718FD0643F4D000B10F27002055
:1024E00068613846CEE70000940100200079054974
:1024F00000EBC00001EB80004069002800D0012003
:1025000070470000940100202DE9F047044600794F
:10251000274900EBC00001EB800720684FF000095D
:10252000C0F80095786880B120682249C0F8081387
:1025300020680121000B40B200F01F0291404009C9
:10254000800000F1E020C0F880112068D0F80C2550
:10255000D0F81485D0F80865D0F810554FF0FF3149
:10256000C0F80C15C0F814152068C0F80815C0F89C
:102570001015501C02D01046FFF777F8B8F1FF3F56
:1025800002D04046FFF771F8681C02D02846FFF7DA
:102590006CF8701C02D03046FFF767F82068FFF730
:1025A000EDFC87F82090C7F80490BDE8F0870000A4
:1025B000940100201003020010B50C46017A052991
:1025C00008D0407A38B1084808A102682046FEF7D2
:1025D000F5FE00E01AB106A12046FEF7EFFE204608
:1025E000BDE81040FEF7F7BE8C0000202573000008
:1025F0000D0A000038B5C3880D46044633B114A057
:10260000009015A216A12846FEF7D8FE217A0529CA
:102610001CD0607A48B1A088FFF762F9164951F8DA
:10262000202016A12846FEF7C9FEA0880021FFF74A
:102630006DFB03461049207A143951F8202001B06F
:102640002846BDE830400EA1FEF7B8BE38BD0000F8
:102650001B5B306D000000001B5B313B33316D00B4
:1026600025734C6F67732064726F707065642028E7
:1026700025642925730D0A008C00002025730000B5
:102680003C25733E2025733A200000000349884210
:1026900001D103487047002070470000002000402F
:1026A0001C00002070B5012670044FF0E0210025C9
:1026B000C1F88001084C4010C4F84803C4F808036E
:1026C00066602F20FFF72AFCA660044C2F20A5602F
:1026D000FFF724FCA57070BD00100140240000200D
:1026E00070B5054688690C4600284FF48471284669
:1026F0000AD0FFF7FCFBD5F81805626AE168885438
:10270000606A401C606270BDFFF7F1FBD5F81805E8
:1027100070BD1FB501238DF80030CDE90121D0E94E
:102720000012684690471FBD1FB501238DF8003089
:102730008DF808100192D0E90012684690471FBD3D
:1027400070B50D4C0020D2B22070201D0B4D0378C7
:10275000EB5C1BB1001DFFF781FE02E00C30FFF7C0
:1027600083FD08B1FEF710F96078002802D02178C7
:102770000029FAD070BD00003C00002010000020AD
:1027800070B5124901200870114C032511A1208851
:1027900005EB0040FFF72AFA0C48083000780028C3
:1027A00013D0208810A105EB0040FFF71FFA07485F
:1027B0000830FDF7DBFD82B22088044905EB0040BC
:1027C000BDE870400831FFF7BDB970BD00000020C2
:1027D000CC0000205472616E7366657220636F6D69
:1027E000706C657465642E0020526563656976655A
:1027F000643A000000B585B00A4601788DF80010F3
:1028000041680191017A8DF80810C1680391007C3C
:102810008DF81000044850F822100C3850F822208F
:102820006846904705B000BDDC0000202DE9F84364
:10283000044610681E4615460F464FF0000810B1BA
:10284000FFF774FBF8B1A86810B1FFF76FFBD0B1C8
:10285000D5E90001C4F84405C4F84815D5E90201DA
:10286000C4F83405C4F838154FF48C754046C4F8E4
:102870001881D4F818110091F2074FF0010107D028
:10288000C4F8501506E087F81D801020BDE8F883D5
:10289000C4F85005B20702D5C4F8401501E0C4F8E9
:1028A0004005300700D42161386848B146F3800004
:1028B000401C4FF0400014D0C4F804030020E5E7AA
:1028C00029462046FFF709FB0028F9D0F87FFF28AA
:1028D000F4D0B97F11B1FEF712FFEFE7FEF716FF54
:1028E000ECE7C4F80803E9E72DE9F84F204D9246DC
:1028F000894606469846012269461846AF68FEF7A3
:102900003BF958B3009800210446801C09E000BF41
:1029100000EA07035AF8212005EB8303401C491CF9
:10292000DA604145F4D34FEA164AFEF7E1F94AEA84
:102930000041601C384005EB80003C4005EB840200
:10294000C160D06866F3C50068F3891069F39F2001
:1029500020F00300401C20F00400D06095F8200413
:1029600002E000BFFEF7E2FF0028FBD1BDE8F88FD0
:10297000C40300202DE9F84F1D4C00256846D4E91A
:1029800001A6FEF7BFF9002738B30023009A61685B
:102990001CE0D1F800C00846944503D9ACEB020214
:1029A0000A6015E0A2EB0C0263440760D0F80CC08B
:1029B000C1698146BCF1000F08D006EB030828F07E
:1029C0007F48C0E9018CC9F81C5005460029E0D1B8
:1029D00028466160FEF770FA03E02846FEF76CFABD
:1029E00010B15046FEF72EF9E770BDE8F88F0000F1
:1029F000240000200D4B10B5596831B102680C68F5
:102A0000A24204D8A21A0A60C161586010BD0B46E8
:102A100003E00B46C969121B21B10C689442F8D33C
:102A2000A41A0C600260C161D86110BD24000020AE
:102A30002DE9F041144E77683D462C4603E0844270
:102A400004D02546E469002CF9D11BE0D4B1A5429D
:102A50000BD1F869706040B90C49012088600021F1
:102A6000B160F0702F20FFF759FA2168E069E86142
:102A700010B10268114401607068874202D00120E1
:102A8000BDE8F0810020FBE7240000200010014099
:102A90002DE9F041194D6C68002C2CD01848002706
:102AA0000068A968B846401A20F07F462068B04206
:102AB0000CD82146361A0744E469087C20B181F815
:102AC0001080886949698847002CEFD12978687897
:102AD000814206D1401CC0B26870022801D185F83D
:102AE0000180064869780C3040F82170BDE8F0415B
:102AF0001420FDF71DBDBDE8F0810000240000207A
:102B00000415014070B50C4605464FF48E71FFF771
:102B1000EEF9216AA068415C206A401C2062C5F879
:102B20001C1570BD1FB500228DF800200291816830
:102B300001914261D0E90012684690471FBD000034
:102B40001FB50A4601788DF8001041680191017A9D
:102B50008DF80810C0680390044850F82210001F38
:102B600050F82220684690471FBD00001800002042
:102B700001490120087070473C00002010B588B062
:102B8000044620220E496846FDF7CCFB0620009043
:102B9000C01F0190029003904FF0EB7006900CB1B3
:102BA000084A00E0002269460748FEF7D3FB08B157
:102BB000FDF7EAFE0448001F447008B010BD000095
:102BC000442F0000712B0000400000202DE9FF473A
:102BD0000C4605464FF40071FFF78FF901274FF4BB
:102BE0000178002618B34FF4927949462846FFF73A
:102BF00079F9E0B149462846FFF779F9C5F8088325
:102C000094F8290000B96F6002208DF80000D5F813
:102C10008004C5F880040390A0690290E0680190E8
:102C2000A661E661D4E900126846904728E00421D5
:102C30002846FFF762F918B34FF484712846FFF76E
:102C400051F9E8B121462846FFF74AFD616AA069BB
:102C5000884215D1E06938B1E268616AA0612069F3
:102C6000E6616662E06008E094F8290000B96F60F0
:102C7000C5F80883A661E268616A2046FFF749FD4E
:102C80004FF48E7841462846FFF72CF978B1206A38
:102C90006169884202D294F8280020B34146284650
:102CA000FFF725F9616911B12046FFF73BFF4FF4AB
:102CB000A27841462846FFF715F9002818D041466A
:102CC0002846FFF714F994F8290000B12F60A06995
:102CD00000280DD0A661E268616A04B02046BDE814
:102CE000F047FFF716BD21462846FFF70BFFDEE74A
:102CF000BDE8FF871FB50A4601788DF800104168CE
:102D00000191017A8DF80810C0680390044850F8CA
:102D10002210001F50F82220684690471FBD000077
:102D2000180000202DE9FF410C464FF4927705462C
:102D30003946FFF7E8F80026C0B139462846FFF7C4
:102D4000E7F802208DF80000D5F88004C5F880046B
:102D50000390D5F83C058DF80800E0680190A66165
:102D6000E661D4E900126846904723E04FF4887783
:102D700039462846FFF7C7F8E0B139462846FFF73D
:102D8000C7F8D5F83C15A069884213D1E06960B155
:102D9000E268D5F8000220F02000C5F80002E069E2
:102DA000A0612069E661E06001E0A661E26820467A
:102DB000FFF7BAFC4FF4A27739462846FFF7A3F88D
:102DC00060B139462846FFF7A3F8A06930B1A66183
:102DD000D5F83C152046E268FFF7A6FC4FF4907743
:102DE00039462846FFF78FF8002813D03946284681
:102DF000FFF78EF8606900280CD0D5F84C058DF8E7
:102E000000608DF80800A06801906661D4E90012A6
:102E100068469047BDE8FF812DE9F05F8346DDE914
:102E20000A4A994690460D460846012703E000BF2E
:102E3000B0FBF8F07F1C4045FAD2B94500D94F46A7
:102E40005FEACA7012D18CB15FEA8A7002D5B9F11B
:102E5000000F01D0202607E0302605E03146584615
:102E6000641EFDF7CDFE0CB1A742F7D35FF001065B
:102E7000B9F1010F02D9A9F1010903E0B5FBF6F0A0
:102E8000404502D306FB08F6F2E7DFF83C9000BFAE
:102E9000B5FBF6F000FB165519F800105846FDF783
:102EA000AFFEB6FBF8F6002EF2D15FEACA7009D089
:102EB000002C07D0A74205D220215846641EFDF7FA
:102EC0009FFEF5E7BDE8F09F262F00000000000000
:102ED0000338FDD8704700000000000000300040BB
:102EE0000000000001000000FFFFFFFF07FF0000DF
:102EF0000000004000000000111213140D0E0F100E
:102F0000FFFFFFFF0007FF0000000040000000007F
:102F1000000000506D05000085210000E123000045
:102F20000338FDD8704730313233343536373839CD
:102F30004142434445460000C91800009D18000066
:102F400095180000FFFFFFFFFFFFFFFFFFFFFFFFE0
:102F5000FFFFFFFF00000000000000000000D6019E
:102F60000701000000404040404040404040414197
:102F7000414141404040404040404040404040404E
:102F800040404040400502020202020202020202E8
:102F900002020202022020202020202020202002E5
:102FA0000202020202029090909090901010101075
:102FB0001010101010101010101010101010101011
:102FC00002020202020288888888888808080808A5
:102FD0000808080808080808080808080808080871
:102FE0000202020240000000652F00007761726E4D
:102FF000696E670064656275670000001B5B313BAA
:1030000033306D001B5B306D000000001B5B313BFB
:1030100033316D001B5B313B33326D001B5B313B49
:1030200033336D001B5B313B33346D001B5B313B35
:1030300033356D001B5B313B33366D001B5B313B21
:1030400033376D00696E666F000000006572726F45
:10305000720000004750494F544500005052530041
:103060005350494D000000005541525400000000EB
:10307000554152544500000062616C6C6F632E6CC8
:103080006F675F6D656D706F6F6C000061707000D1
:103090000031000000000020D0000000EC0800001B
:1030A000D0310000D000002018270000FC080000EC
:1030B00054300000000000005C3000000000000000
:1030C00060300000000000006830000000000000D8
:1030D00070300000000000007830000000000003A5
:1030E0008C30000000000303680000206000002016
:1030F0006800002004030020C80000201800000021
:10310000004E6F7264696300000000000000000060
:1031100000000000000000000000000000000000AF
:10312000000000000000000000000000000000009F
:10313000000000000000000000000000000000008F
:1031400000000000002000400000000000200040BF
:1031500000000000382F0000000000000000000008
:10316000000000000000000000000000000000005F
:103170000000000000000000000000004C300000D3
:10318000EC2F000044300000F42F00000430000059
:10319000FC2F00000C300000143000001C30000038
:1031A000243000002C300000343000003C3000009F
:1031B0000090D003000000000000000000000000AC
:1031C00000000000000000000000000000000000FF
:0400000500000201F4
:00000001FF
